:020000040000FA
:08000000FF23831690002D2858
:08000800B800030EB9000C1052
:1000100005190D28301431100F28311430101C3000
:10002000DE22AF002F1D28282F1C1C283008013A83
:10003000B0003108013AB1000C30DE22AC002C1CBB
:100040002828301C26288512051628280512851612
:10005000390E8300B80E380E09008501073099006B
:1000600083169F010F3085000C148312013090001D
:100070000B178B178501B5014022A201A301A40132
:10008000A501A601A701A001A1010519582805197C
:100090005A2800302002031945280730200203188F
:1000A0005E28A10A0C30210203196128A00145280D
:1000B0000000000000000000A00A4528A001A101E6
:1000C0004528A001A10105197128051973280030E0
:1000D0002002031963280730200203187728A001A3
:1000E00063280000000000000000A00A63288E01C1
:1000F0008F01A001A101A11505198F2805199128CB
:100100000030200203197C280730200203189528AC
:10011000A20D2214A10B8D289928A0017C28000093
:10012000000000000000A00A7C28A20D2210A10BF4
:100130008D28A001A1010519A9280519AB280030B7
:10014000200203199B28073020020318AF28A001C2
:100150003C280000000000000000A00A9B28A0012D
:10016000A101A1150519C5280519C72800302002CD
:100170000319B228073020020318CB28A30D23143B
:10018000A10BC328CF28A001B22800000000000066
:100190000000A00AB228A30D2310A10BC328A001C0
:1001A000A1010519DF280519E128003020020319F3
:1001B000D128073020020318E528A0013C280000C0
:1001C000000000000000A00AD128A001A101A11593
:1001D0000519FB280519FD28003020020319E8281D
:1001E0000730200203180129A40D2414A10BF928BB
:1001F0000529A001E8280000000000000000A00A76
:10020000E828A40D2410A10BF928A001A1010519CB
:10021000152905191729003020020319072907306D
:10022000200203181B29A001A729000000000000DC
:100230000000A00A0729A001A101A1150519312973
:10024000051933290030200203191E290730200226
:1002500003183729A50D2514A10B2F293B29A0012F
:100260001E290000000000000000A00A1E29A50DA4
:100270002510A10B2F29A001A10105194B29051952
:100280004D290030200203193D29073020020318B0
:100290005129A001A7290000000000000000A00AC9
:1002A0003D29A001A101A115051967290519692991
:1002B00000302002031954290730200203186D2949
:1002C000A60D2614A10B65297129A001542900004F
:1002D000000000000000A00A5429A60D2610A10B62
:1002E0006529A001A101051981290519832900307B
:1002F0002002031973290730200203188729A0015F
:10030000A7290000000000000000A00A7329A00136
:10031000A101A11505199D2905199F290030200269
:1003200003198A29073020020318A329A70D2714CF
:10033000A10B9B29A729A0018A2900000000000029
:100340000000A00A8A29A70D2710A10B9B292208CB
:1003500023062406250626062706031D3C28220917
:10036000031DB429B5013C2822080319C72AA21B82
:10037000C9297039703A03195E2AB5011C30DE2292
:10038000AF00AF1A3C280030DE222206031D3C28B5
:10039000E329B5011C30DE22AF00AF1E3C28220845
:1003A000193E03183C281030DE222206031D3C288B
:1003B0001130DE222306031D3C282408A300250853
:1003C000A4002608A5002308E039B700203A031945
:1003D000212A3708803A0319352A3708E03A0319E9
:1003E000512A3708003A0319C72A3708403A031937
:1003F000022A3708603A0319022A3708A03A03197B
:100400004D2A3C281C30DE22AF002F1C0A2A23086C
:10041000203AA300AF18192A231E162AA31E132A56
:1004200085160512182A05168512182A0512851236
:100430002316A31A1E2A301431103C283114301010
:100440003C283F302302031D3C281C30DE22AF0035
:100450002F1C2D2A2408FF3AA400A41B322A301492
:1004600031103C28311430103C281C30DE22AF0003
:10047000AF1C3C28231E3210231A321440223C2881
:10048000321C4A2A311C472A851605120800051617
:1004900085120800051285120800A31E502A3C2868
:1004A0003C28EC302302031D3C28073024060319A6
:1004B000E92A2508B6002408CE223A28351CBD2991
:1004C000A5080319842A2208743A03196C2A220801
:1004D0007C3A0319742A3C282308DE222402031DD7
:1004E0003C28B50104233C2807302306031D7D2A40
:1004F00008302406031D012BED2A2408B60023082A
:10050000CE22B50104233C28221D952AA2183C289E
:10051000221CB22A8B2A2308B300B3030310B30DA5
:100520000310B30DB51404233C28B51C3C28220845
:1005300003393307B400073034060319E42AA21D37
:10054000A92A2308B6003408CE22B401B501042339
:100550003C283408DE222302031D3C28B401B501E7
:1005600004233C28B51C3C28A21DBE2A2308B60043
:100570001C30CE22B301B50104233C281C30DE22FE
:100580002302031D3C28B301B50104233C282208A3
:100590002306031D3C28351485013C2883169B0047
:1005A0008312360883169A001C1555309D00AA3018
:1005B0009D009C149C18DA2A8312080083169B0065
:1005C0001C141A088312080008302306031D012B8F
:1005D000ED2A08302506031D3C280330B600003004
:1005E000CE220130B6000C30CE22C030B600103022
:1005F000CE228030B6001130CE220230B6001C3040
:10060000CE22B30135103A28FF308500142314237D
:10061000142314231423142385010800000002303E
:10062000BA00BA0B112B08004730BB000E23182B61
:10063000BB0B162B000008003C30BC001423BC0B85
:040640001E2B080065
:04064400003400344A
:02400E00843FED
:104200000300000000000000FF0000001F001D0070
:104210000400000000000000010000000000000099
:10422000C00080000000000000000000000000004E
:10423000000000000000000002000000000000007C
:10424000000000000000000000000000000000006E
:10425000000000000000000000000000000000005E
:04426000000000005A
:00000001FF
